:103000000C942A180C9445180C9445180C944518E7
:103010000C9445180C9445180C9445180C944518BC
:103020000C9445180C9445180C9445180C944518AC
:103030000C9445180C9445180C9445180C9445189C
:103040000C9445180C9445180C9445180C9445188C
:103050000C94451811241FBECFE5D4E0DEBFCDBFD0
:1030600010E0A0E6B0E0E4E3F4E302C005900D92C6
:10307000A036B107D9F711E0A0E6B0E001C01D927B
:10308000AE32B107E1F70C942C1C0C94001859C017
:10309000C79A2BE02A95F1F7C79826E02A95F1F711
:1030A00008951BE019B918E11AB908955D9BFECF88
:1030B0004CB908955F9BFECF4CB108952FEF2A9530
:1030C000F1F71A95D9F70895332718E080E0331FF8
:1030D00010F4C59A01C0C598880FB6998160D8DFF1
:1030E0001A95A9F7382F089500001FEB17BBC79852
:1030F000C19A1FEFE3DFC1981FEFE0DF3CEAE5DF95
:1031000033E5E3DF003280F0002372F0A0E2DCDF81
:10311000333561F030E0D9DFBBDF3CEAD6DF33E5A1
:10312000D4DFAA95A1F702C030E0CFDF30E0CDDFD9
:1031300010E1C4DF0895EAEEF9E1EE0FFF1F3BD185
:1031400008951FE51DBF11271BBF1FEF12BBBB9AC0
:10315000C398C19A18BB12E017BBA3DFABDF4B319A
:10316000E9F3443519F4A6DF042F19C1433511F4EE
:10317000E2DFF4CF463529F443E398DF44E396DFFA
:10318000EDCF453429F416E011BD1EE011BD07C195
:10319000463729F441E38ADF40E388DFDFCF443755
:1031A00069F4EEEEF9E1EE0FFF1F0DD1412D4F3F17
:1031B00011F07CDFFACF442779DFD0CF403719F404
:1031C00043E574DFCBCF413619F449E56FDFC6CF55
:1031D000483719F46FDFC398E2C0493719F46ADF42
:1031E000C39ADDC02F93EEEEF9E1EE0FFF1FEBD097
:1031F000212D2F3F29F0201709F0F9CF2F9102C080
:103200002F91CAC0403511F46FDFC9C0433471F447
:1032100051DF38E45ADF362F58DF352F56DF342F91
:1032200054DF11E02227510F621F0BC0433671F4A7
:1032300041DF30E44ADF362F48DF352F46DF342FB9
:1032400044DF222011F410E239DFA9C0423599F49D
:1032500038E23BDF362F39DF352F37DF35DF432FBD
:1032600025DF30E232DF362F30DF352F2EDF2CDF47
:10327000432F1CDF24C0413429F41CDF642F1ADFE4
:10328000542F8DC0443481F415DF30EC1EDF362F0F
:103290001CDF352F1ADF342F18DF10E20FDF11E0AB
:1032A0002227510F621F7BC0443671F430EA0DDFD4
:1032B000362F0BDF352F09DF07DF432FF7DE11E055
:1032C0002227510F621F4ACF4C3421F412E017BB62
:1032D000C19A65C0453659F43CEAF7DE30E8F5DEC0
:1032E00034E0F3DE30E0F1DE10E3E8DE58C04C36C7
:1032F00071F4E0DE3CEAE9DE342F3670306EE5DE54
:1033000030E0E3DE30E0E1DE10E3D8DE48C04337F2
:1033100089F4B2E005D0B1E003D0B0E001D01ECF17
:1033200030E3D3DE30E0D1DE3B2FCFDECDDE432FE6
:10333000BDDE08954D3659F43CE4C7DE362FC5DEB8
:10334000352FC3DE30E0C1DE1FEFB8DE28C04A33C0
:1033500059F4B0DEC42FAEDED42FACDE742F442778
:1033600010D01FEFABDE1BC04E32B1F4A3DEC42F72
:10337000A1DED42F9FDE742F9DDE03D01FEF9EDED3
:103380000EC03C2FA2DE3D2FA0DE372F9EDE342F55
:103390009CDE482F8BDE08954FE388DEDFCE4DE0C4
:1033A00085DEDCCE0000133029F0000000001A9505
:1033B0001330E9F70895C895402D403019F076DEB6
:1033C0003196F9CF0895C895102C3196C895202CC8
:1033D0003196089541565220495350001000110073
:1033E00012001300200028003000340038003A0199
:1033F0003B014101420143014401450146014800AE
:103400004C005500560058005C005E0160016101EF
:103410006401650166016701680069016C00700064
:1034200071007250730174017501760177017801A2
:043430007901FFFF20
:023800002BC0DB
:103804008BE089B988E18AB986E880BD0895F0E043
:10381400E0E0099408955F9BFECF8CB19927089549
:103824005D9BFECF8CB9089581E40E94121C86E54D
:103834000E94121C82E50E94121C82E40E94121C47
:103844008FE40E94121C8FE40E94121C84E50E94E3
:10385400121C0895CFE5D4E0DEBFCDBF1124EE24C1
:10386400FF246701F89481E085BF82E085BFA698B4
:10387400AE9ABB9A0E94021C8EB581608EBD8EB535
:1038840084608EBD1DBC1CBCC0E0D0E027E2C0310A
:10389400D20731F488B398E0892788BBC0E0D0E030
:1038A40021969E9909C0C39A15BA81E085BF15BEB9
:1038B4001EBCAE980E9447185F9B03C08CB1833531
:1038C400A9F08CB59DB5805C984A00F3C39A15BAEB
:1038D40081E085BF15BE1EBC9E9B04C0AE980E94AD
:1038E400091CD4CFAE980E944718D0CFC39A1EBCEF
:1038F4000E94161C0E940D1C99278635910509F417
:103904006FC08735910594F58534910509F431C16B
:10391400863491059CF48B31910509F434C18C31C2
:1039240091051CF4892B31F337C18134910509F4D5
:103934005FC08334910509F4BDC02EC18235910561
:1039440009F483C0833591054CF48C34910509F452
:1039540063C08035910509F45FC01EC183359105AC
:1039640039F28435910509F440C016C18D369105AC
:1039740009F4C3C08E369105A4F48336910509F485
:1039840093C08436910524F48136910511F104C164
:103994008436910509F44AC08536910509F4C2C0FC
:1039A400FBC084379105B9F0853791053CF4803725
:1039B400910569F08337910589F1EEC08837910547
:1039C40009F4CFC08937910509F4CFC0E5C083E578
:1039D400E4C089E5E2C084E70E94121C80E0DDC0F7
:1039E40081E30E94121C80E3D8C00E940D1C14C005
:1039F4000E940D1C9927182F00270E940D1C99273F
:103A0400802B912B90932A0180932901880F991F71
:103A140090932D0180932C018DE0BFC082E00E9421
:103A2400121C84E90E94121C8EE1B7C08091290106
:103A34008EBB8091290190912A01892F99278FBBF0
:103A4400E199FECFE09A8DB3A8C0C114D10461F00E
:103A540080912C0190912D018C159D0529F489EB01
:103A64000E94121C89E014C007B600FCFDCF81E15E
:103A740080935700E895E0912C01F0912D01319647
:103A840084910E94121CE0912C01F0912D018491EB
:103A94000E94121C80912C0190912D01029690930A
:103AA4002D0180932C0126CFC3980E940D1CE82E73
:103AB400FF24B2CF0E940D1C9927982F8827E82A4B
:103AC400F92A89E0E81689EBF80631F4EE24FF249C
:103AD400C0902C01D0902D01C39A07B600FCFDCFF5
:103AE40021E080912C0190912D010701FC0120938C
:103AF4005700E895112402968BCF8091290190916B
:103B04002A018050984108F087CF07B600FCFDCF0A
:103B140025E080912C0190912D01FC012093570008
:103B2400E8957ACF10922A011092290143E020E00F
:103B340030E0F90140935700E89507B600FCFDCF4B
:103B4400C90180589F4F9C0157E18138950788F33C
:103B540090932A018093290181E180935700E8958D
:103B64005BCF0E940D1CC39857CF0E940D1CC39AB3
:103B740053CF88E190E028E00FB6F894A89581BD72
:103B84000FBE21BD49CF10922D0110922C0110922D
:103B94002A0110922901AECE8FE30E94121CAACEF4
:0400000300003000C9
:00000001FF
